:020000040000FA
:0400000068303A2802
:040004000034003490
:08000800A000030EA100831209
:1000100081018B100B11210E8300A00E200E090010
:0C007400203084008001840A80300402E7
:10008000031C3C28352183160C308505870183121B
:10009000850187010730990000309A0010308316DF
:1000A0008E008312603083168F0083120030831617
:1000B000910000008312C830831681008312313012
:1000C0009000003083168C00831210308B00BD1B13
:1000D0006F2885196F286400851D6B2868213D1CD9
:1000E0007228522181018E018F010B118B100B1090
:1000F0008C018B178E20321990201721B40B8C287D
:10010000031085190314BA0DF0303A020319642163
:100110000F303A02031960218E217A28640008000A
:10012000080032110130B7008B13203037078316D7
:100130009B001C141A088312A40010303707831682
:100140009B001C141A088312A30000303707831683
:100150009B001C141A088312A2008B17331CB628AC
:1001600022090339A200A309A409A5090130370215
:10017000031DBF283E18BF283E143F1446210130FE
:100180003702031DC8283E1CC8283E103F144921D1
:10019000C928B70A02303702031808009428013032
:1001A000B600B400B500B70085018701B213512134
:1001B0008E20B40BE828031085190314BA0DF03013
:1001C0003A0203190629B50BE8289630B50012212A
:1001D000321DD8283211331CF2282D090339AD0005
:1001E000AE09AF098B1320303707BC002F08BB00C6
:1001F000202110303707BC002E08BB002021003022
:100200003707BC002D08BB0020218B178501870113
:10021000B70AB6010130B50002303702031CD828F6
:10022000522108000130370203194D2108003F1CFC
:1002300008003F101030BC003E08BB002021080021
:100240008B133B0883161C159A0083123C088316F7
:100250009B0055309D00AA309D009C1464009C18A2
:100260002E291C1183128B170800831600309B0067
:100270001C141A088312BD003D1C080083161030A0
:100280009B001C141A088312BE0008000130BE0037
:10029000080087010530D40008000508333A8500BE
:1002A00008000800BE013E14080001303E02031998
:1002B0005A2908000130D40056150730D300080031
:1002C0003E143F14462108003E103F144921080007
:1002D000B601B401B5013D1C7029BD01BD147229E0
:1002E000BD013D143D08B6006400762977297829C0
:1002F00079297A293330B51B8500B51F8501B40BE8
:100300007429B50B74290310B60CB608031D7429A3
:100310000030BC003D08BB00202108008F080319F5
:1003200008008E018F01D0080319DE29D00FAB29F8
:1003300056180516D618851656190514D61985149B
:10034000D60158180512D818851258190510D81951
:100350008510D801DE295008D10056180516D61888
:10036000851656190514D619851451080E0203185E
:10037000C52958180512D818851258190510D8190A
:100380008510FF305002031908008F08031D080074
:100390008E2051080E02031CC52956180512D618C6
:1003A000851256190510D619851058180516D81833
:1003B000851658190514D819851408000030530201
:1003C000031DF7293E18EF29051A58140130051AA4
:1003D000D000851AD8140130851AD00008000130E9
:1003E000D40056140130D0000130D3000800051AA3
:1003F000FD295614851AD814FF29D6145814013033
:10040000D000D40B080001305302031D112AD61569
:100410000530D4000230D3003E180800D601D301C5
:10042000080002305302031D232A56158714D815DD
:100430000330D4000330D3003E1808008701D601F2
:10044000D301D815080003305302031D332A871443
:1004500007150330D4000430D3003E18080087018C
:10046000D3015815080004305302031D442A871491
:10047000071507140330D4000530D3003E180800D8
:100480008701D3015815080005305302031D562A71
:1004900087140715071487160330D4000630D300DD
:1004A0003E1808008701D301581508000630530292
:1004B000031D692A871407150714871607160330CA
:1004C000D4000730D3003E1808008701D301581527
:1004D000080007305302031D7D2A871407150714EF
:1004E0008716071687150130D4000730D3003E1851
:1004F00008008701D301581508000030D300080018
:084000000700030007000100A6
:02400E00CC33B1
:104200000100FF00FF00FF00FF00FF00FF00FF00B4
:10421000FF00FF00FF00FF00FF00FF00FF00FF00A6
:104220000100FF00FF00FF00FF00FF00FF00FF0094
:10423000FF00FF00FF00FF00FF00FF00FF00FF0086
:104240000100FF00FF00FF00FF00FF00FF00FF0074
:10425000FF00FF00FF00FF00FF00FF00FF00050060
:10426000FF00FF00FF00FF00FF00FF00FF00FF0056
:10427000FF00FF00FF00FF00FF00FF00FF00FF0046
:10428000FF00FF00FF00FF00FF00FF00FF00FF0036
:10429000FF00FF00FF00FF00FF00FF00FF00FF0026
:1042A000FF00FF00FF00FF00FF00FF00FF00FF0016
:1042B000FF00FF00FF00FF00FF00FF00FF00FF0006
:1042C000FF00FF00FF00FF00FF00FF00FF00FF00F6
:1042D000FF00FF00FF00FF00FF00FF00FF00FF00E6
:1042E000FF00FF00FF00FF00FF00FF00FF00FF00D6
:1042F000FF00FF00FF00FF00FF00FF00FF000000C5
:00000001FF
